:100000000C9445000C946D000C946D000C946D00E4
:100010000C946D000C946D000C946D000C946D00AC
:100020000C946D000C946D000C946D000C946D009C
:100030000C946D000C946D000C946D000C946D008C
:100040000C94ED050C946D000C9410080C9442086F
:100050000C946D000C946D000C946D000C946D006C
:100060000C946D000C946D0072756E2D6272696453
:1000700067650A000A000A00EE03C105C905D0053C
:10008000D705E2057208FB08C50511241FBECFEF96
:10009000D8E0DEBFCDBF11E0A0E0B1E0EAE2F8E1D8
:1000A00002C005900D92A437B107D9F722E0A4E76A
:1000B000B1E001C01D92A635B207E1F710E0C8E833
:1000C000D0E004C02297FE010E94D40AC837D107AD
:1000D000C9F70E940B090C94080C0C94000026E050
:1000E00040E950ED63E070E080917D0190917E01E8
:1000F0000E94AE0784E791E00E94E7028FE791E05B
:100100000E94AE058FE791E00E9412058823D1F38B
:1001100062E171E08FE791E00C949E096091060125
:100120008FE791E00E942B046EE271E08FE791E08F
:100130000E94810960910601709107014AE050E038
:100140008FE791E00E94530A66E371E08FE791E048
:100150000E948109609106017091070140E150E021
:100160008FE791E00E94530A6EE371E08FE791E020
:100170000E948109609106017091070148E050E0FA
:100180008FE791E00E94530A66E471E08FE791E007
:100190000E948109609106017091070142E050E0E0
:1001A0008FE791E00E945B0A809106019091070120
:1001B0008E37910529F48FE791E00E94D404FFCF98
:1001C000019690930701809306010895FC01238115
:1001D00034812627022E2295207F2025032E322FC0
:1001E00022952F700226269532272327220F220FD1
:1001F000220F2025FC01348323830895CF93DF93BE
:10020000EC018D819E81DC01ED91FC916C8101906E
:10021000F081E02D09958D819E81DC01ED91FC91AD
:100220000190F081E02D6B81DF91CF9109948F9245
:100230009F92AF92BF92CF92DF92EF92FF92CF93B5
:10024000DF93EC016B010E9437064B015C01E12C4E
:10025000F12C8D819E81DC01ED91FC910680F7816E
:10026000E02D099597FF0DC00E943706681979099E
:100270008A099B096C157D058E059F0550F38FEF4C
:100280009FEFDF91CF91FF90EF90DF90CF90BF90E5
:10029000AF909F908F900895CF93DF93EC018D8165
:1002A0009E81DC01ED91FC910480F581E02D0995A2
:1002B0001816190654F48D819E81DC01ED91FC9194
:1002C0000680F781E02D0995EACFDF91CF9108955F
:1002D0002F923F924F925F926F927F928F929F9256
:1002E000AF92BF92CF92DF92EF92FF920F931F9344
:1002F000CF93DF93CDB7DEB72D970FB6F894DEBF5F
:100300000FBECDBF3C011B013C832B832701BF8265
:10031000AE827801EC0CFD1CE40EF51EFD82AF2CC4
:10032000B12CCA01860F971F99878887D901A00F22
:10033000B11FBB87AA87F601E40DF51DFD87EC8789
:10034000F3018085B81608F027C1EFEFFFEFD30166
:100350001496FC93EE93139715968D919C91169796
:10036000DC01ED91FC910190F081E02D6FEF09959A
:100370006FEFC3010E94E600F30185819681DC01E5
:10038000ED91FC910190F081E02DD3016C910995E4
:10039000F3016081C3010E94E600D30115968D919F
:1003A0009C911697DC01ED91FC910190F081E02D7C
:1003B0006D8109956A2DC3010E94E600F3018581D4
:1003C0009681DC01ED91FC910190F081E02D6E2D84
:1003D00009956E2DC3010E94E6006101888599850B
:1003E000C816D906A1F0F301858196818601DC014A
:1003F000ED91FC910190F081E02DD6016D916D01A0
:100400000995F8016081C3010E94E600E7CFCB8027
:10041000DC808A859B85C816D906B1F0D301159674
:100420008D919C9116978601DC01ED91FC910190D4
:10043000F081E02DD6016D916D010995F801608183
:10044000C3010E94E600E5CF62018C859D85C81638
:10045000D906B1F0D30115968D919C91169786011E
:10046000DC01ED91FC910190F081E02DD6016D91C0
:100470006D010995F8016081C3010E94E600E5CF96
:10048000C3010E94FE0064E670E0C3010E941701F0
:100490008F3F910509F075C0EFEFFFEFD301149680
:1004A000FC93EE9313976FEFC3010E94E60065E0A3
:1004B00070E0C3010E941701D3016C91262F30E038
:1004C0008217930709F05DC0C3010E94E6006AE04D
:1004D00070E0C3010E9417018C0197FD52C0682F84
:1004E000C3010E94E6006AE070E0C3010E941701A8
:1004F0006C0197FD46C0682FC3010E94E6000A8385
:100500001982E981FA81CE0EDF1E00E010E065E07D
:1005100070E0C3010C151D0599F00E94170197FDAD
:100520000CC00815190528F4EE81FF81E00FF11FBA
:100530008083682FC3010E94E6000F5F1F4FE7CF43
:100540000E9417016C0197FD1CC065E070E0C301BB
:100550000E94170197FD15C0DC2CCC24C80ED91EB3
:10056000D30113968D919C9114978C159D0549F498
:100570008C918F5F8C93C8018016910678F4C4012A
:100580000DC0B39464E670E080E090E00E946606DF
:10059000C3010E944C01D4CE8FEF9FEF2D960FB672
:1005A000F894DEBF0FBECDBFDF91CF911F910F91A9
:1005B000FF90EF90DF90CF90BF90AF909F908F9083
:1005C0007F906F905F904F903F902F9008953F9253
:1005D0004F925F926F927F928F929F92AF92BF9253
:1005E000CF92DF92EF92FF920F931F93CF93DF93FF
:1005F000CDB7DEB72E970FB6F894DEBF0FBECDBFD6
:100600003C01DC0117968C9117978111CFC081E0D6
:1006100017968C93C3010E944C0168EE73E080E052
:1006200090E00E946606F30185819681DC01ED91E0
:10063000FC910480F581E02D09951816190654F3F4
:1006400045E0542E4424439452E3352EE8E0F1E093
:10065000DE011696852D01900D928A95E1F7F30142
:100660004086812C912CA12CB12CC12CD12CE12CB9
:10067000F12C00E010E020E030E045E050E0BE0169
:100680006A5F7F4FC3010E94680163E0D301159642
:100690008D919C9116970E9483096AEF70E080E02B
:1006A00090E00E94660666E770E0F301858196811E
:1006B0000E945C096AEF70E080E090E00E946606AC
:1006C00064E770E0D30115968D919C9116970E9476
:1006D0005C0964EF71E080E090E00E94660668E6E5
:1006E00070E0F301858196810E945C0964EF71E0FE
:1006F00080E090E00E946606C3010E944C01EDE09C
:10070000F1E0DE011196852D01900D928A95E1F7B9
:10071000D30118963C9234E0832E912CFE013B9637
:100720005F0120E030E045E050E0BE016F5F7F4FA9
:10073000C3010E9468018F3FFFEF9F0739F468EE05
:1007400073E080E090E00E94660680CF2B85211147
:10075000FFCF049711F52C8530E02053310944E692
:10076000429FC001439F900D11242D8530E02053FE
:1007700031096AE0629FA001639F500D1124840F2C
:10078000951F2E8530E020533109820F931FD3012E
:1007900012969C938E93119705C084E690E0F30126
:1007A0009283818382E3D30118968C932E960FB6A1
:1007B000F894DEBF0FBECDBFDF91CF911F910F9197
:1007C000FF90EF90DF90CF90BF90AF909F908F9071
:1007D0007F906F905F904F903F90089510927401BA
:1007E0008FEA91E090937A018093790110927B01D6
:1007F00010927C0190937E0180937D0108958F92E9
:100800009F92AF92BF92CF92DF92EF92FF920F939F
:100810001F9348015901C12CD12CE12CF12C00E08F
:1008200010E020E030E00E9468011F910F91FF90DE
:10083000EF90DF90CF90BF90AF909F908F900895F2
:100840000F931F9300E010E020E030E00E94FF03D0
:100850001F910F910895CF93DF9300D0CDB7DEB7EE
:10086000DC0152968C915297882389F080E5898328
:100870006A8342E050E0BE016F5F7F4F1C968D910E
:100880009C911D970E94200481E090E01FC0559626
:10089000ED91FC91569753968C91539791E0980F58
:1008A00053969C935397E80FF11D608353969C9148
:1008B000539754968C915497981308C0ED91FC91DE
:1008C00011970284F385E02DCD0109950F900F90CB
:1008D000DF91CF910895AF92BF92CF92DF92EF92C6
:1008E000FF920F931F93CF93DF9300D0CDB7DEB766
:1008F0005C017A01DC0152968C91811104C08B015C
:10090000E60EF71E41C06A01BFEFCB1ADB0AC60133
:1009100069837A830E941A098C01FC0180E5819326
:10092000A70169817A81CF010E94FF0BA601B8015E
:10093000F501848595850E9420040115110519F0A3
:10094000C8010E941C09C70122C0D5015596ED912E
:10095000FC91569753968C91539791E0980F53962C
:100960009C93D8019D918D01E80FF11D9083F501B5
:1009700093898489981308C00190F081E02D028446
:10098000F385E02DC50109950E151F05F1F60F90B1
:100990000F90DF91CF911F910F91FF90EF90DF901B
:1009A000CF90BF90AF900895CF93DF93EC018A89E9
:1009B00081110AC04B8950E06D897E898C859D85A7
:1009C0000E94200481E08B8BDF91CF910895FC0180
:1009D0001382128248EE53E060E070E04483558356
:1009E0006683778382E591E09183808384E791E059
:1009F0009587848716861786118A108A81E0828BF4
:100A00000895CF93DF93EC018A89811108C08D8905
:100A10009E89009711F00E941C0981E08A8BDF916A
:100A2000CF9108950F931F93CF93DF931F92CDB76C
:100A3000DEB721E6298301E010E09E012F5F3F4FE2
:100A400041E050E0B901FC01848595850E94FF03D7
:100A500081E09981913009F080E00F90DF91CF9192
:100A60001F910F910895EF92FF920F931F93CF93D1
:100A7000DF9300D0CDB7DEB77C01FC018685811104
:100A800014C0178680E7898380E28A8320893189B0
:100A900000E210E042E050E0BE016F5F7F4F8485CE
:100AA00095850E94FF03F70186870F900F90DF91D5
:100AB000CF911F910F91FF90EF900895CF93DF9307
:100AC000EC010E9433058E8590E0DF91CF9108956F
:100AD000CF93DF93EC010E9433058E85882369F064
:100AE00081508E87E889F9898F8591E0980F9F87DB
:100AF000E80FF11D808190E002C08FEF9FEFDF9142
:100B0000CF910895CF93DF93EC010E9433058E853A
:100B1000882341F08F85E889F989E80FF11D8081EC
:100B200090E002C08FEF9FEFDF91CF910895CF93B8
:100B3000DF93EC010E94010588899989009721F0D3
:100B40000E941C09198A188ADF91CF91089522E525
:100B500031E0FC01318320830C949705CF93DF9320
:100B6000EC018C859D850E94E702CE010E949705CD
:100B700080E290E00E941A09998B888BDF91CF91D7
:100B800008958FE791E00C94E7048FE791E00C94CF
:100B9000A70584E791E090939701809396010895CB
:100BA00084E791E0909399018093980108950F93C1
:100BB00000E020E040E060E08AE991E00E94EF0878
:100BC0000F9108950F9300E020E040E060E080EA9C
:100BD00091E00E94EF080F9108951F920F920FB6B7
:100BE0000F9211242F933F938F939F93AF93BF93B3
:100BF0008091A7019091A801A091A901B091AA01AB
:100C00003091A60123E0230F2D3720F40196A11D7A
:100C1000B11D05C026E8230F0296A11DB11D20932A
:100C2000A6018093A7019093A801A093A901B09376
:100C3000AA018091AB019091AC01A091AD01B0915E
:100C4000AE010196A11DB11D8093AB019093AC0143
:100C5000A093AD01B093AE01BF91AF919F918F91E1
:100C60003F912F910F900FBE0F901F9018952FB7A7
:100C7000F8946091A7017091A8018091A9019091C9
:100C8000AA012FBF08953FB7F8948091AB019091CE
:100C9000AC01A091AD01B091AE0126B5A89B05C0F5
:100CA0002F3F19F00196A11DB11D3FBF6627782F78
:100CB000892F9A2F620F711D811D911D42E0660FD1
:100CC000771F881F991F4A95D1F70895CF92DF9219
:100CD000EF92FF92CF93DF936B017C010E9443065A
:100CE000EB01C114D104E104F10489F00E94870AE8
:100CF0000E9443066C1B7D0B683E734090F381E0BD
:100D0000C81AD108E108F108C851DC4FEACFDF91D9
:100D1000CF91FF90EF90DF90CF900895789484B5B5
:100D2000826084BD84B5816084BD85B5826085BDE7
:100D300085B5816085BDEEE6F0E0808181608083CD
:100D4000E1E8F0E0108280818260808380818160B0
:100D50008083E0E8F0E0808181608083E1EBF0E077
:100D6000808184608083E0EBF0E08081816080831B
:100D7000EAE7F0E080818460808380818260808304
:100D80008081816080838081806880831092C1002F
:100D90000895FC01818D228D90E0805C9F4F821B25
:100DA000910960E470E00E94880A0895FC01918D29
:100DB000828D981731F0828DE80FF11D858D90E0BE
:100DC00008958FEF9FEF0895FC01918D828D981704
:100DD00061F0828DDF01A80FB11D5D968C91928D1F
:100DE0009F5F9F73928F90E008958FEF9FEF08951C
:100DF00088E698E0892B49F080E090E0892B29F083
:100E00000E94680881110C9400000895FC01848DF3
:100E1000DF01A80FB11DA35ABF4F2C91848D90E024
:100E200001968F739927848FA689B7892C93A089FF
:100E3000B1898C9180648C93938D848D981306C0B6
:100E40000288F389E02D80818F7D80830895CF9380
:100E5000DF93EC01888D8823C9F0EA89FB898081C2
:100E600085FD05C0A889B9898C9186FD0FC00FB694
:100E700007FCF5CF808185FFF2CFA889B9898C91D5
:100E800085FFEDCFCE010E940607E7CFDF91CF911E
:100E90000895CF92DF92FF920F931F93CF93DF932A
:100EA0001F92CDB7DEB76C01DC015B969C915B971E
:100EB0005C968C915C97981307C05096ED91FC91CD
:100EC0005197808185FD32C0F601038D10E00F5FE0
:100ED0001F4F0F731127F02EF601848DF81211C0E9
:100EE0000FB607FCF9CFD6015096ED91FC915197C2
:100EF000808185FFF1CFC60169830E940607698161
:100F0000EBCF838DE80FF11DE35AFF4F6083D601CD
:100F10005B960C935B975296ED91FC915397808171
:100F20008062808381E058968C930DC0D6015696DE
:100F3000ED91FC91579760835096ED91FC915197FC
:100F400080818064808381E090E00F90DF91CF9179
:100F50001F910F91FF90DF90CF900895BF92CF9295
:100F6000DF92EF92FF92CF93DF93EC016A017B0156
:100F7000B22EE889F98982E08083411581EE580715
:100F800061057105A1F060E079E08DE390E0A701D3
:100F900096010E949C0A2150310941095109569538
:100FA000479537952795211580E1380798F0E8890E
:100FB000F989108260E874E88EE190E0A70196015B
:100FC0000E949C0A215031094109510956954795C3
:100FD00037952795EC85FD853083EE85FF85208349
:100FE000188EEC89FD89B082EA89FB898081806155
:100FF0008083EA89FB89808188608083EA89FB8914
:10100000808180688083EA89FB8980818F7D8083ED
:10101000DF91CF91FF90EF90DF90CF90BF90089538
:101020001F920F920FB60F9211242F938F939F93BD
:10103000EF93FF93E091BF01F091C0018081E091B7
:10104000C501F091C60182FD12C090818091C80156
:101050008F5F8F732091C901821751F0E091C80111
:10106000F0E0E155FE4F958F8093C80101C080816B
:10107000FF91EF919F918F912F910F900FBE0F9045
:101080001F9018951F920F920FB60F9211242F9355
:101090003F934F935F936F937F938F939F93AF9300
:1010A000BF93EF93FF938FEA91E00E940607FF91B1
:1010B000EF91BF91AF919F918F917F916F915F91D0
:1010C0004F913F912F910F900FBE0F901F90189549
:1010D0008FEA91E00E94C90621E0892B09F420E003
:1010E000822F08951092B2011092B10188EE93E020
:1010F000A0E0B0E08093B3019093B401A093B50158
:10110000B093B60182E691E09093B0018093AF0175
:1011100085EC90E09093BC018093BB0184EC90E05F
:101120009093BE018093BD0180EC90E09093C0014C
:101130008093BF0181EC90E09093C2018093C10144
:1011400082EC90E09093C4018093C30186EC90E020
:101150009093C6018093C5011092C8011092C901F5
:101160001092CA011092CB010895AF92BF92CF9214
:10117000DF92EF92FF920F931F93CF93DF936C0157
:101180007B01C0E0D0E000E010E0F601EC0FFD1FB5
:101190004AE050E06281C7010E94800A5C016EE271
:1011A000C7010E9483098A0D9B1D080F191F2196F4
:1011B000C330D10551F74AE050E0F6016581C7011F
:1011C0000E94800A800F911FDF91CF911F910F9194
:1011D000FF90EF90DF90CF90BF90AF9008950F9366
:1011E000FC0182E791E091838083628343832483BF
:1011F00005830F91089582E791E090934D028093CB
:101200004C0210924E0210924F0210925002109215
:101210005102089508950E948E060E940A090E94B4
:101220006F00C8EFD6E00E948E002097E1F30E9485
:10123000F806F9CF0C94D80A0C94700BCF92DF9279
:10124000EF92FF920F931F93CF93DF936C017A017C
:10125000EB01E60EF71E00E010E0CE15DF0561F0B1
:101260006991D601ED91FC910190F081E02DC601CC
:101270000995080F191FF1CFC801DF91CF911F9178
:101280000F91FF90EF90DF90CF9008956115710559
:1012900081F0DB010D900020E9F7AD0141505109CB
:1012A000461B570BDC01ED91FC910280F381E02D90
:1012B000099480E090E00895EF92FF920F931F93BE
:1012C000CF93DF938C01FB01C0E0D0E064917F01FC
:1012D0008FEFE81AF80A662361F0D801ED91FC91CE
:1012E0000190F081E02DC8010995C80FD91FF701C1
:1012F000EDCFCE01DF91CF911F910F91FF90EF9035
:1013000008950C944609DC01ED91FC910190F08167
:10131000E02D09940F931F93CF93DF93EC016DE0C1
:101320000E9483098C016AE0CE010E948309800F2C
:10133000911FDF91CF911F910F9108950F931F93EC
:10134000CF93DF93EC010E9446098C01CE010E94ED
:101350008A09800F911FDF91CF911F910F910895FE
:101360008F929F92AF92BF92CF92DF92EF92FF92B5
:101370000F931F93CF93DF93CDB7DEB7A1970FB62F
:10138000F894DEBF0FBECDBF7C01C42EE52FCB018C
:10139000D22E19A221E02D1510F02AE0D22E8E01B6
:1013A0000F5D1F4F8D2C912CA12CB12C6C2D7E2FFD
:1013B000A50194010E949C0A8C2DD29E80191124B3
:1013C000015011098A3014F4805D01C0895CF80174
:1013D0008083211531054105510521F0C22EE32FEF
:1013E000CA01E4CFB801C7010E944609A1960FB611
:1013F000F894DEBF0FBECDBFDF91CF911F910F914B
:10140000FF90EF90DF90CF90BF90AF909F908F9024
:101410000895CF92DF92EF92FF920F931F93CF9395
:10142000DF93EC016A017B012115310579F4E88134
:10143000F9810190F081E02D642FDF91CF911F9110
:101440000F91FF90EF90DF90CF9009942A303105F3
:10145000E9F477FF1AC06DE20E9483098C014427EA
:101460005527BA014C195D096E097F092AE0CE01A2
:101470000E94B009800F911FDF91CF911F910F91B2
:10148000FF90EF90DF90CF9008952AE0B701A6017A
:10149000CE01DF91CF911F910F91FF90EF90DF90E0
:1014A000CF900C94B0099A01AB01662757FD609567
:1014B000762F0C94090A0F931F93CF93DF93EC01BF
:1014C0009A01AB01662757FD6095762F0E94090AA5
:1014D0008C01CE010E948A09800F911FDF91CF916C
:1014E0001F910F9108952115310541F4DC01ED9113
:1014F000FC910190F081E02D642F09940C94B009C7
:101500009A01462F50E060E070E00C94730A089551
:1015100097FB072E16F4009407D077FD09D00E94A0
:10152000BE0A07FC05D03EF4909581959F4F089523
:10153000709561957F4F0895A1E21A2EAA1BBB1BDF
:10154000FD010DC0AA1FBB1FEE1FFF1FA217B3078F
:10155000E407F50720F0A21BB30BE40BF50B661FA5
:10156000771F881F991F1A9469F760957095809569
:1015700090959B01AC01BD01CF010895AA1BBB1B37
:1015800051E107C0AA1FBB1FA617B70710F0A61B83
:10159000B70B881F991F5A95A9F780959095BC01A4
:1015A000CD010895EE0FFF1F0590F491E02D0994F1
:1015B000CF93DF938230910510F482E090E0E091C8
:1015C0005402F091550220E030E0A0E0B0E0309706
:1015D00039F14081518148175907B8F04817590728
:1015E00071F482819381109729F013969C938E93C6
:1015F00012972CC0909355028093540227C0211556
:10160000310531F04217530718F0A901DB0101C081
:10161000EF019A01BD01DF010280F381E02DD7CFF8
:1016200021153105F9F0281B390B2430310580F4E0
:101630008A819B816115710521F0FB01938382836F
:1016400004C09093550280935402FE01329644C028
:10165000FE01E20FF31F81939193225031093983E8
:1016600028833AC02091520230915302232B41F437
:1016700020910201309103013093530220935202D2
:1016800020910001309101012115310541F42DB760
:101690003EB74091040150910501241B350BE091A8
:1016A0005202F0915302E217F307A0F42E1B3F0BF6
:1016B0002817390778F0AC014E5F5F4F24173507C4
:1016C00048F04E0F5F1F5093530240935202819394
:1016D000919302C0E0E0F0E0CF01DF91CF91089557
:1016E000CF93DF93009709F487C0FC0132971382F0
:1016F0001282C0915402D0915502209781F420812A
:101700003181280F391F8091520290915302821724
:10171000930779F5F0935302E09352026DC0DE0116
:1017200020E030E0AE17BF0750F412964D915C9167
:1017300013979D014115510509F1DA01F3CFB383E8
:10174000A28340815181840F951F8A179B0771F4F2
:101750008D919C911197840F951F029691838083A0
:1017600012968D919C911397938382832115310555
:1017700029F4F0935502E09354023EC0D901139628
:10178000FC93EE9312974D915D91A40FB51FEA174C
:10179000FB0779F480819181840F951F0296D9010E
:1017A00011969C938E938281938113969C938E9332
:1017B0001297E0E0F0E08A819B81009719F0FE012A
:1017C000EC01F9CFCE01029628813981820F931F57
:1017D00020915202309153022817390769F430974B
:1017E00029F4109255021092540202C01382128200
:1017F000D0935302C0935202DF91CF910895FB0121
:10180000DC0102C001900D9241505040D8F708957C
:1018100010E0C8E8D0E004C0FE010E94D40A22967D
:0A182000CA38D107C9F7F894FFCFCA
:10182A00000056028000210058585858585858311C
:10183A0030304153434949205461626C65207E200F
:10184A00436861726163746572204D6170002C2077
:10185A006465633A20002C206865783A20002C20C1
:10186A006F63743A20002C2062696E3A20000000EF
:10187A0000002B046B045E0568058205D404000091
:10188A00000049071E09C906E406D6062707000014
:04189A000000B5088D
:107E0000112484B714BE81FFF0D085E080938100F7
:107E100082E08093C00088E18093C10086E0809377
:107E2000C20080E18093C4008EE0C9D0259A86E02C
:107E300020E33CEF91E0309385002093840096BBD3
:107E4000B09BFECF1D9AA8958150A9F7CC24DD24C4
:107E500088248394B5E0AB2EA1E19A2EF3E0BF2EE7
:107E6000A2D0813461F49FD0082FAFD0023811F036
:107E7000013811F484E001C083E08DD089C08234E0
:107E800011F484E103C0853419F485E0A6D080C0E4
:107E9000853579F488D0E82EFF2485D0082F10E0AE
:107EA000102F00270E291F29000F111F8ED06801E7
:107EB0006FC0863521F484E090D080E0DECF843638
:107EC00009F040C070D06FD0082F6DD080E0C81688
:107ED00080E7D80618F4F601B7BEE895C0E0D1E017
:107EE00062D089930C17E1F7F0E0CF16F0E7DF06D8
:107EF00018F0F601B7BEE89568D007B600FCFDCFD4
:107F0000A601A0E0B1E02C9130E011968C91119780
:107F100090E0982F8827822B932B1296FA010C0160
:107F200087BEE89511244E5F5F4FF1E0A038BF0790
:107F300051F7F601A7BEE89507B600FCFDCF97BE46
:107F4000E89526C08437B1F42ED02DD0F82E2BD052
:107F50003CD0F601EF2C8F010F5F1F4F84911BD097
:107F6000EA94F801C1F70894C11CD11CFA94CF0C13
:107F7000D11C0EC0853739F428D08EE10CD085E9AC
:107F80000AD08FE07ACF813511F488E018D01DD067
:107F900080E101D065CF982F8091C00085FFFCCF94
:107FA0009093C60008958091C00087FFFCCF809118
:107FB000C00084FD01C0A8958091C6000895E0E648
:107FC000F0E098E1908380830895EDDF803219F02E
:107FD00088E0F5DFFFCF84E1DECF1F93182FE3DFCA
:107FE0001150E9F7F2DF1F91089580E0E8DFEE27F6
:047FF000FF270994CA
:027FFE00040479
:0400000300007E007B
:00000001FF
